BL51 BANKED LINKER/LOCATER V6.05                                                        08/17/2015  16:42:11  PAGE 1


BL51 BANKED LINKER/LOCATER V6.05, INVOKED BY:
C:\KEIL\C51\BIN\BL51.EXE clockdingshi.obj TO sz RAMSIZE (256)


MEMORY MODEL: SMALL


INPUT MODULES INCLUDED:
  clockdingshi.obj (CLOCKDINGSHI)
  C:\KEIL\C51\LIB\C51S.LIB (?C_STARTUP)
  C:\KEIL\C51\LIB\C51S.LIB (?C_INIT)


LINK MAP OF MODULE:  sz (CLOCKDINGSHI)


            TYPE    BASE      LENGTH    RELOCATION   SEGMENT NAME
            -----------------------------------------------------

            * * * * * * *   D A T A   M E M O R Y   * * * * * * *
            REG     0000H     0008H     ABSOLUTE     "REG BANK 0"
            DATA    0008H     001DH     UNIT         ?DT?CLOCKDINGSHI
            DATA    0025H     0006H     UNIT         _DATA_GROUP_
            IDATA   002BH     0001H     UNIT         ?STACK

            * * * * * * *   C O D E   M E M O R Y   * * * * * * *
            CODE    0000H     0003H     ABSOLUTE     
            CODE    0003H     0007H     UNIT         ?C_INITSEG
                    000AH     0001H                  *** GAP ***
            CODE    000BH     0003H     ABSOLUTE     
            CODE    000EH     0257H     UNIT         ?PR?MAIN?CLOCKDINGSHI
            CODE    0265H     00FCH     UNIT         ?PR?KEYSCAN?CLOCKDINGSHI
            CODE    0361H     008CH     UNIT         ?C_C51STARTUP
            CODE    03EDH     0069H     UNIT         ?PR?KEYSCAN0?CLOCKDINGSHI
            CODE    0456H     0068H     UNIT         ?PR?_DISPLAY?CLOCKDINGSHI
            CODE    04BEH     001AH     UNIT         ?PR?_DELAY?CLOCKDINGSHI
            CODE    04D8H     0013H     UNIT         ?PR?TIME0?CLOCKDINGSHI
            CODE    04EBH     0010H     UNIT         ?CO?CLOCKDINGSHI



OVERLAY MAP OF MODULE:   sz (CLOCKDINGSHI)


SEGMENT                             DATA_GROUP 
  +--> CALLED SEGMENT             START    LENGTH
-------------------------------------------------
?C_C51STARTUP                     -----    -----
  +--> ?PR?MAIN?CLOCKDINGSHI
  +--> ?C_INITSEG

?PR?MAIN?CLOCKDINGSHI             -----    -----
  +--> ?PR?KEYSCAN0?CLOCKDINGSHI
  +--> ?PR?KEYSCAN?CLOCKDINGSHI
  +--> ?PR?_DISPLAY?CLOCKDINGSHI

?PR?KEYSCAN0?CLOCKDINGSHI         -----    -----
  +--> ?PR?_DELAY?CLOCKDINGSHI
BL51 BANKED LINKER/LOCATER V6.05                                                      08/17/2015  16:42:11  PAGE 2



?PR?KEYSCAN?CLOCKDINGSHI          -----    -----
  +--> ?PR?_DELAY?CLOCKDINGSHI

?PR?_DISPLAY?CLOCKDINGSHI         0025H    0006H
  +--> ?CO?CLOCKDINGSHI
  +--> ?PR?_DELAY?CLOCKDINGSHI



SYMBOL TABLE OF MODULE:  sz (CLOCKDINGSHI)

  VALUE           TYPE          NAME
  ----------------------------------

  -------         MODULE        CLOCKDINGSHI
  C:0000H         SYMBOL        _ICE_DUMMY_
  D:0080H         PUBLIC        P0
  D:00A0H         PUBLIC        P2
  D:00B0H         PUBLIC        P3
  B:00A8H.7       PUBLIC        EA
  D:0008H         PUBLIC        baoshijieshu
  D:0009H         PUBLIC        miao10
  C:04EBH         PUBLIC        table
  D:000AH         PUBLIC        miao20
  D:000BH         PUBLIC        a0
  C:04C4H         PUBLIC        _delay
  D:000CH         PUBLIC        b0
  D:000DH         PUBLIC        a1
  D:000EH         PUBLIC        c0
  D:000FH         PUBLIC        b1
  D:0010H         PUBLIC        c1
  D:0011H         PUBLIC        fen10
  D:0012H         PUBLIC        fen20
  B:00A0H.3       PUBLIC        beep
  C:03EDH         PUBLIC        keyscan0
  C:000EH         PUBLIC        main
  D:0013H         PUBLIC        shi10
  D:0014H         PUBLIC        shi20
  B:00A0H.6       PUBLIC        dula
  B:00A0H.7       PUBLIC        wela
  D:0089H         PUBLIC        TMOD
  D:0015H         PUBLIC        temp
  D:0016H         PUBLIC        wei
  B:00A8H.1       PUBLIC        ET0
  D:0017H         PUBLIC        key
  D:008CH         PUBLIC        TH0
  D:0018H         PUBLIC        yidingshi
  D:008AH         PUBLIC        TL0
  B:0088H.4       PUBLIC        TR0
  D:0019H         PUBLIC        ok
  D:001AH         PUBLIC        pp
  C:04D8H         PUBLIC        time0
  D:001CH         PUBLIC        qq
  D:001DH         PUBLIC        f
  D:001EH         PUBLIC        change
  D:001FH         PUBLIC        j
BL51 BANKED LINKER/LOCATER V6.05                                                      08/17/2015  16:42:11  PAGE 3


  D:0020H         PUBLIC        dingshi
  D:0021H         PUBLIC        k
  D:0022H         PUBLIC        m
  C:0265H         PUBLIC        keyscan
  D:0023H         PUBLIC        s
  D:0024H         PUBLIC        baoshi
  C:0456H         PUBLIC        _display
  C:04BEH         SYMBOL        L?0110
  -------         PROC          L?0109
  -------         ENDPROC       L?0109
  C:04BEH         SYMBOL        L?0110
  -------         PROC          _DELAY
  D:0007H         SYMBOL        i
  C:04C4H         LINE#         43
  C:04C4H         LINE#         44
  C:04C4H         LINE#         45
  C:04CDH         LINE#         46
  C:04D7H         LINE#         47
  -------         ENDPROC       _DELAY
  -------         PROC          _DISPLAY
  D:0007H         SYMBOL        shi2
  D:0005H         SYMBOL        shi1
  D:0003H         SYMBOL        fen2
  D:0028H         SYMBOL        fen1
  D:0029H         SYMBOL        miao2
  D:002AH         SYMBOL        miao1
  C:0456H         LINE#         48
  C:0456H         LINE#         49
  C:0456H         LINE#         50
  C:0458H         LINE#         51
  C:045FH         LINE#         52
  C:0461H         LINE#         53
  C:0463H         LINE#         55
  C:0465H         LINE#         56
  C:0468H         LINE#         57
  C:0468H         LINE#         58
  C:0468H         LINE#         59
  C:046BH         LINE#         61
  C:0471H         LINE#         62
  C:0473H         LINE#         63
  C:0475H         LINE#         65
  C:0478H         LINE#         66
  C:0478H         LINE#         67
  C:0478H         LINE#         68
  C:047BH         LINE#         70
  C:047FH         LINE#         71
  C:0481H         LINE#         72
  C:0483H         LINE#         74
  C:0486H         LINE#         75
  C:0486H         LINE#         76
  C:0486H         LINE#         77
  C:0489H         LINE#         79
  C:0490H         LINE#         80
  C:0492H         LINE#         81
  C:0494H         LINE#         83
  C:0497H         LINE#         84
  C:0497H         LINE#         85
BL51 BANKED LINKER/LOCATER V6.05                                                      08/17/2015  16:42:11  PAGE 4


  C:0497H         LINE#         86
  C:049AH         LINE#         88
  C:049FH         LINE#         89
  C:04A1H         LINE#         90
  C:04A3H         LINE#         92
  C:04A6H         LINE#         93
  C:04A6H         LINE#         94
  C:04A6H         LINE#         95
  C:04A9H         LINE#         97
  C:04AEH         LINE#         98
  C:04B0H         LINE#         99
  C:04B2H         LINE#         101
  C:04B5H         LINE#         102
  C:04B7H         LINE#         103
  C:04B9H         LINE#         104
  -------         ENDPROC       _DISPLAY
  -------         PROC          KEYSCAN0
  C:03EDH         LINE#         107
  C:03EDH         LINE#         108
  C:03EDH         LINE#         109
  C:03F0H         LINE#         110
  C:03F3H         LINE#         111
  C:03F6H         LINE#         112
  C:03FCH         LINE#         113
  C:03FCH         LINE#         114
  C:0401H         LINE#         115
  C:0407H         LINE#         116
  C:0407H         LINE#         117
  C:040AH         LINE#         118
  C:0414H         LINE#         119
  C:0414H         LINE#         120
  C:0414H         LINE#         121
  C:0417H         LINE#         122
  C:041AH         LINE#         123
  C:041CH         LINE#         125
  C:041CH         LINE#         126
  C:041FH         LINE#         127
  C:0422H         LINE#         128
  C:0424H         LINE#         129
  C:0424H         LINE#         130
  C:0424H         LINE#         132
  C:0424H         LINE#         133
  C:0424H         LINE#         134
  C:0427H         LINE#         135
  C:042AH         LINE#         136
  C:042DH         LINE#         137
  C:0433H         LINE#         138
  C:0433H         LINE#         139
  C:0438H         LINE#         140
  C:043EH         LINE#         141
  C:043EH         LINE#         142
  C:0441H         LINE#         143
  C:044BH         LINE#         144
  C:044BH         LINE#         145
  C:044BH         LINE#         146
  C:044EH         LINE#         147
  C:0451H         LINE#         148
BL51 BANKED LINKER/LOCATER V6.05                                                      08/17/2015  16:42:11  PAGE 5


  C:0452H         LINE#         149
  C:0452H         LINE#         150
  C:0455H         LINE#         151
  C:0455H         LINE#         152
  C:0455H         LINE#         154
  C:0455H         LINE#         155
  C:0455H         LINE#         156
  -------         ENDPROC       KEYSCAN0
  -------         PROC          KEYSCAN
  C:0265H         LINE#         159
  C:0265H         LINE#         160
  C:0265H         LINE#         161
  C:0265H         LINE#         162
  C:0268H         LINE#         163
  C:026BH         LINE#         164
  C:026EH         LINE#         165
  C:0274H         LINE#         166
  C:0274H         LINE#         167
  C:0279H         LINE#         168
  C:027FH         LINE#         169
  C:027FH         LINE#         170
  C:0282H         LINE#         171
  C:0294H         LINE#         172
  C:0294H         LINE#         173
  C:0294H         LINE#         174
  C:0297H         LINE#         175
  C:0299H         LINE#         176
  C:029BH         LINE#         178
  C:029BH         LINE#         179
  C:029EH         LINE#         180
  C:02A0H         LINE#         181
  C:02A2H         LINE#         183
  C:02A2H         LINE#         184
  C:02A5H         LINE#         185
  C:02A7H         LINE#         186
  C:02A9H         LINE#         188
  C:02A9H         LINE#         189
  C:02ACH         LINE#         190
  C:02AEH         LINE#         191
  C:02AEH         LINE#         192
  C:02AEH         LINE#         193
  C:02B4H         LINE#         194
  C:02B4H         LINE#         195
  C:02B7H         LINE#         196
  C:02BAH         LINE#         197
  C:02BCH         LINE#         198
  C:02BEH         LINE#         199
  C:02C0H         LINE#         200
  C:02C0H         LINE#         201
  C:02C0H         LINE#         202
  C:02C3H         LINE#         203
  C:02C6H         LINE#         204
  C:02C9H         LINE#         205
  C:02CFH         LINE#         206
  C:02CFH         LINE#         207
  C:02D4H         LINE#         208
  C:02DAH         LINE#         209
BL51 BANKED LINKER/LOCATER V6.05                                                      08/17/2015  16:42:11  PAGE 6


  C:02DAH         LINE#         210
  C:02DDH         LINE#         211
  C:02EFH         LINE#         212
  C:02EFH         LINE#         213
  C:02EFH         LINE#         214
  C:02F2H         LINE#         215
  C:02F4H         LINE#         216
  C:02F6H         LINE#         218
  C:02F6H         LINE#         219
  C:02F9H         LINE#         220
  C:02FBH         LINE#         221
  C:02FDH         LINE#         223
  C:02FDH         LINE#         224
  C:0300H         LINE#         225
  C:0302H         LINE#         226
  C:0304H         LINE#         228
  C:0304H         LINE#         229
  C:0307H         LINE#         230
  C:0309H         LINE#         231
  C:0309H         LINE#         232
  C:0309H         LINE#         233
  C:030FH         LINE#         234
  C:030FH         LINE#         235
  C:0312H         LINE#         236
  C:0315H         LINE#         237
  C:0317H         LINE#         238
  C:0319H         LINE#         239
  C:031BH         LINE#         240
  C:031BH         LINE#         241
  C:031BH         LINE#         242
  C:031EH         LINE#         243
  C:0321H         LINE#         244
  C:0324H         LINE#         245
  C:032AH         LINE#         246
  C:032AH         LINE#         247
  C:032FH         LINE#         248
  C:0335H         LINE#         249
  C:0335H         LINE#         250
  C:0338H         LINE#         251
  C:0342H         LINE#         252
  C:0342H         LINE#         253
  C:0342H         LINE#         254
  C:0345H         LINE#         255
  C:0347H         LINE#         256
  C:0349H         LINE#         258
  C:0349H         LINE#         259
  C:034CH         LINE#         260
  C:034EH         LINE#         261
  C:034EH         LINE#         262
  C:034EH         LINE#         263
  C:0354H         LINE#         264
  C:0354H         LINE#         265
  C:0357H         LINE#         266
  C:035AH         LINE#         267
  C:035CH         LINE#         268
  C:035EH         LINE#         269
  C:0360H         LINE#         270
BL51 BANKED LINKER/LOCATER V6.05                                                      08/17/2015  16:42:11  PAGE 7


  C:0360H         LINE#         271
  C:0360H         LINE#         272
  C:0360H         LINE#         273
  -------         ENDPROC       KEYSCAN
  -------         PROC          MAIN
  C:000EH         LINE#         275
  C:000EH         LINE#         276
  C:000EH         LINE#         277
  C:0011H         LINE#         279
  C:0014H         LINE#         280
  C:0017H         LINE#         281
  C:0019H         LINE#         282
  C:001BH         LINE#         284
  C:001BH         LINE#         285
  C:001EH         LINE#         287
  C:0024H         LINE#         288
  C:0026H         LINE#         289
  C:0028H         LINE#         291
  C:0030H         LINE#         292
  C:0034H         LINE#         293
  C:0036H         LINE#         294
  C:003BH         LINE#         295
  C:003BH         LINE#         296
  C:003EH         LINE#         297
  C:0040H         LINE#         298
  C:0045H         LINE#         299
  C:0045H         LINE#         300
  C:0048H         LINE#         301
  C:004AH         LINE#         302
  C:004FH         LINE#         303
  C:004FH         LINE#         304
  C:0052H         LINE#         305
  C:0052H         LINE#         306
  C:0052H         LINE#         307
  C:0052H         LINE#         308
  C:0052H         LINE#         310
  C:005BH         LINE#         311
  C:0063H         LINE#         312
  C:006CH         LINE#         313
  C:0074H         LINE#         314
  C:007DH         LINE#         315
  C:0085H         LINE#         316
  C:0093H         LINE#         317
  C:0096H         LINE#         319
  C:0096H         LINE#         320
  C:009FH         LINE#         321
  C:00A1H         LINE#         322
  C:00A4H         LINE#         323
  C:00AAH         LINE#         324
  C:00AAH         LINE#         326
  C:00C0H         LINE#         327
  C:00C0H         LINE#         328
  C:00C7H         LINE#         329
  C:00CCH         LINE#         331
  C:00CEH         LINE#         332
  C:00D0H         LINE#         333
  C:00E9H         LINE#         334
BL51 BANKED LINKER/LOCATER V6.05                                                      08/17/2015  16:42:11  PAGE 8


  C:00EBH         LINE#         336
  C:00F2H         LINE#         337
  C:00F5H         LINE#         338
  C:00F7H         LINE#         339
  C:00FEH         LINE#         340
  C:0103H         LINE#         342
  C:0105H         LINE#         343
  C:0107H         LINE#         344
  C:010CH         LINE#         345
  C:0113H         LINE#         346
  C:0118H         LINE#         348
  C:011AH         LINE#         349
  C:011CH         LINE#         350
  C:011FH         LINE#         351
  C:011FH         LINE#         352
  C:0122H         LINE#         353
  C:0122H         LINE#         354
  C:012CH         LINE#         355
  C:0136H         LINE#         356
  C:0140H         LINE#         357
  C:0152H         LINE#         358
  C:0152H         LINE#         359
  C:015BH         LINE#         360
  C:015BH         LINE#         361
  C:015DH         LINE#         362
  C:016FH         LINE#         363
  C:0172H         LINE#         364
  C:0178H         LINE#         365
  C:0178H         LINE#         366
  C:018EH         LINE#         367
  C:018EH         LINE#         368
  C:0195H         LINE#         369
  C:019AH         LINE#         371
  C:019CH         LINE#         372
  C:019EH         LINE#         373
  C:01B7H         LINE#         374
  C:01BCH         LINE#         376
  C:01C3H         LINE#         377
  C:01C6H         LINE#         378
  C:01C8H         LINE#         379
  C:01CFH         LINE#         380
  C:01D4H         LINE#         382
  C:01D6H         LINE#         383
  C:01D8H         LINE#         384
  C:01DDH         LINE#         385
  C:01E4H         LINE#         386
  C:01E9H         LINE#         388
  C:01EBH         LINE#         389
  C:01EDH         LINE#         390
  C:01F0H         LINE#         391
  C:01F0H         LINE#         392
  C:01F3H         LINE#         393
  C:01F3H         LINE#         394
  C:01F6H         LINE#         395
  C:0208H         LINE#         396
  C:0208H         LINE#         397
  C:0208H         LINE#         398
BL51 BANKED LINKER/LOCATER V6.05                                                      08/17/2015  16:42:11  PAGE 9


  C:020DH         LINE#         399
  C:020DH         LINE#         400
  C:022BH         LINE#         401
  C:022DH         LINE#         402
  C:022DH         LINE#         403
  C:0260H         LINE#         404
  C:0262H         LINE#         405
  -------         ENDPROC       MAIN
  -------         PROC          TIME0
  C:04D8H         LINE#         408
  C:04DAH         LINE#         409
  C:04DDH         LINE#         410
  C:04E0H         LINE#         411
  C:04E8H         LINE#         412
  -------         ENDPROC       TIME0
  -------         ENDMOD        CLOCKDINGSHI

Program Size: data=44.0 xdata=0 code=1274
LINK/LOCATE RUN COMPLETE.  0 WARNING(S),  0 ERROR(S)
